:100000000C9446000C9463000C9463000C94630001
:100010000C9463000C9463000C9463000C946300D4
:100020000C9463000C9463000C9463000C946300C4
:100030000C9463000C9463000C9463000C946300B4
:100040000C947E010C9463000C94B3010C94040294
:100050000C9463000C9463000C9463000C94630094
:100060000C9463000C9463000C9463000C94630084
:100070000C9463000C9463000C94DB010C942B0231
:100080000C9463000C9463000C94630011241FBE55
:10009000CFEFD0E1DEBFCDBF11E0A0E0B1E0EEE2F6
:1000A000F1E100E00BBF02C007900D92AC39B1073F
:1000B000D9F713E0ACE9B1E001C01D92A93BB1074B
:1000C000E1F70C9465000C940000CFEFD0E1DEBFA7
:1000D000CDBFEE24FF240E941D036CE672E086EA89
:1000E00092E00E945303B7018CEC92E00E9453030C
:1000F0008C0180E091E00E941A0486E091E00E9469
:100100001A0480E091E00E941A04B8018EE191E0A7
:100110000E94DD038091650080618093650080917D
:100120006500886080936500C49A81E0E816F10458
:10013000A9F0E2E0EE16F10424F4E114F10431F048
:100140001EC0F2E0EF16F10489F019C0809165003D
:100150008F7E8093650083E491E00BC08091650001
:10016000877F8093650086E491E003C0C49889E4AA
:1001700091E09F938F930E9405040F900F90089435
:10018000E11CF11C83E0E816F10414F0EE24FF24D6
:10019000C0E0D0E00FE911E08C2F0E942501F801AA
:1001A00081938F0199279F938F938CE491E09F9384
:1001B0008F930E9405040F900F900F900F9021963F
:1001C000C830D1054CF383B399279F938F9382E571
:1001D00091E09F938F930E9405040F900F900F90D2
:1001E0000F90C3E6D0E00E94A70190912E0380916A
:1001F0002D03981731F18091AF039091B0030E94C5
:100200009A03182F992787FD90959F938F938BE5DD
:1002100091E09F938F930E9405040F900F900F9091
:100220000F90103271F487E691E00E941A048091D9
:10023000AF039091B0030E949A0383E891E00E947B
:100240001A042197D7FFCFCF65CF97B1907C982B19
:10025000906297B9369A3699FECF85B1992708955D
:10026000009731F0A4E0B0E01197F1F70197D1F7D2
:100270000895009731F0A0EABFE01197F1F70197D8
:10028000D1F70895CF93C82F882331F084E690E00A
:100290000E943001C150D1F7CF910895CF93C82F5C
:1002A000882331F08AE090E00E943001C150D1F7FC
:1002B000CF910895CF93C82F882331F084E690E042
:1002C0000E943901C150D1F7CF910895CF93C82F23
:1002D000882331F08AE090E00E943901C150D1F7C3
:1002E000CF910895CF93C82F882331F081E090E01B
:1002F0000E943901C150D1F7CF9108951F920F92FA
:100300000FB60F9211248F939F9380919E018F5F60
:1003100080939E018A3058F010929E0180919C013A
:1003200090919D01019690939D0180939C0186E0A0
:1003300082BF9F918F910F900FBE0F901F901895C5
:1003400084E083BF12BE81E087BF78940895209136
:100350009C0130919D0180919C0190919D0182179B
:100360009307C9F308951F920F920FB60F921124AD
:100370002F938F939F93EF93FF932CB180912E0334
:1003800090912D03891B803861F080912E03E82F16
:10039000FF27EF77F070E35DFC4F22838F5F809340
:1003A0002E03FF91EF919F918F912F910F900FBE90
:1003B0000F901F9018951F920F920FB60F92112455
:1003C0002F938F939F93EF93FF9320919C008091A5
:1003D000A8019091A701891B803861F08091A80144
:1003E000E82FFF27EF77F070E955FE4F22838F5FEC
:1003F0008093A801FF91EF919F918F912F910F9082
:100400000FBE0F901F9018951F920F920FB60F926C
:1004100011248F939F93EF93FF9390912A028091E1
:100420002902981711F455980DC080912902E82FE0
:10043000FF27EF77F070E75DFD4F8F5F8093290214
:1004400082818CB9FF91EF919F918F910F900FBE98
:100450000F901F9018951F920F920FB60F921124B4
:100460008F939F93EF93FF939091AC028091AB0297
:10047000981731F480919A008F7D80939A000EC076
:100480008091AB02E82FFF27EF77F070E555FD4F25
:100490008F5F8093AB02828180939C00FF91EF91EC
:1004A0009F918F910F900FBE0F901F901895909174
:1004B0002E0380912D039817D1F380912D03E82FFF
:1004C000FF27EF77F070E35DFC4F92818F5F8093A1
:1004D0002D03892F992708950E945702089590911E
:1004E000A8018091A7019817D1F38091A701E82F67
:1004F000FF27EF77F070E955FE4F92818F5F809371
:10050000A701892F992708950E946F020895CF931C
:10051000C82F8A3019F48DE00E94870280912A0248
:1005200090912902891B8038C9F380912A02E82F13
:10053000FF27EF77F070E75DFD4FC2838F5F8093F9
:100540002A02559A80E090E0CF9108950E94870298
:100550000895CF93C82F8A3019F48DE00E94A90224
:100560008091AC029091AB02891B8038C9F38091D5
:10057000AC02E82FFF27EF77F070E555FD4FC283FF
:100580008F5F8093AC0280919A00806280939A0082
:1005900080E090E0CF9108950E94A9020895CF9342
:1005A000DF93EC018881882361F088818A3019F417
:1005B0008DE00E94870289910E94870288818823AA
:1005C000A1F7DF91CF910895CF93DF93EC0188815C
:1005D000882361F088818A3019F48DE00E94A90295
:1005E00089910E94A90288818823A1F7DF91CF9188
:1005F00008950F931F93CF93C62F8C01662339F074
:10060000F80181918F010E948702C150C9F7CF91F3
:100610001F910F9108950F931F93CF93C62F8C01B5
:10062000662339F0F80181918F010E948702C15041
:10063000C9F7CF911F910F9108959FEF9BBB1ABAF5
:1006400098BB80E187BB95BB14BA92BB11BA93B932
:1006500012B810926200109261009093650088E1D8
:100660008093640010BE1092900029E129B91BB854
:1006700098E99AB98EE080939500109298002093A3
:10068000990010929B0090939A0080939D0087ECB4
:1006900086B980E487B986B1877C11F03699FECFA0
:1006A0000E94A00108950F931F93CF93DF938C01B5
:1006B000EB01009711F4672BC1F16EE070E081E06F
:1006C00090E00E940D07FC01892B71F180E8838383
:1006D000209771F0D387C28781E883838091AF032D
:1006E0009091B003892B21F4F093B003E093AF0312
:1006F00001151105C9F0118700878381826083830A
:100700008091B1039091B203892B71F4F093B203FD
:10071000E093B1038091B3039091B403892B21F44A
:10072000F093B403E093B303CF01DF91CF911F9116
:100730000F910895CF93DF93EC014B81842F99277C
:1007400080FF2EC086FF09C04F7B4B838E819F8127
:1007500001969F838E838A812CC082FF11C0E8811D
:10076000F9818081282F332727FD30952115310508
:1007700019F440624B8314C03196F983E88313C0A7
:10078000EA85FB85CE0109959C0197FF0CC08B8102
:1007900099272F5F3F4F11F4806101C080628B83E6
:1007A0008FEF9FEF07C08E819F8101969F838E837D
:1007B000822F9927DF91CF910895EF92FF920F93A7
:1007C0001F93CF93DF93EC018B01EE24FF24FB01F9
:1007D000838181FD03C08FEF9FEF10C08991882333
:1007E00061F0F80120853185B801F9010995892B5F
:1007F000A9F38FEFE82EF82EF1CFC701DF91CF914B
:100800001F910F91FF90EF900895CF93DF93CDB795
:10081000DEB7E5E0F0E0EC0FFD1F81919191AF01B3
:10082000BC018091B1039091B2030E945004DF910A
:10083000CF9108950F931F93CF93DF93EC0100E0C6
:1008400010E0E091B103F091B203838181FD03C018
:100850008FEF9FEF20C08991882371F0E091B10361
:10086000F091B20320853185BF01F9010995892BEB
:1008700091F30FEF1FEFEFCFE091B103F091B203CF
:1008800020853185BF018AE0F9010995892B11F096
:100890000FEF1FEFC801DF91CF911F910F910895C6
:1008A0002F923F924F925F926F927F928F929F9280
:1008B000AF92BF92CF92DF92EF92FF920F931F936E
:1008C000CF93DF93CDB7DEB762970FB6F894DEBF54
:1008D0000FBECDBFEE24FF2487011C017E876D87EC
:1008E0002A01CC24DD24FC01D782C682838181FDCC
:1008F00068C28FEF9FEF78C28D859E8501969E8797
:100900008D87C0FE4BC28F8580538A30D0F49F857F
:10091000903339F4662029F4C3FC03C0E0E0F1E031
:100920008DC08AE0689E602C1124FF856F0E20ED3B
:10093000620E67FE02C05FE7652EC3FC42C2762CE2
:1009400040C2C3FE04C0662011F441E0642EEF856E
:100950008E2F992787FD9095883691058CF58536E1
:1009600091050CF06EC08335910509F493C0843570
:100970009105CCF48B32910509F449C08C32910574
:100980004CF48032910509F446C08332910509F494
:100990004AC0FEC18D32910509F440C08E329105E6
:1009A00009F444C0F5C18336910509F450C084367A
:1009B00091050CF08AC08835910509F4BCC0E8C1E6
:1009C0008037910509F4B1C08137910584F48C36E4
:1009D000910591F18D3691052CF48936910509F434
:1009E00074C0D6C18F36910509F49CC0D1C185373A
:1009F000910509F4A2C08637910524F48337910547
:100A000071F1C6C18837910509F495C0C1C180E173
:100A100090E0C82AD92AE0E2F0E010C080E890E037
:100A2000C82AD92ACEC1E0E4F0E008C088E090E00E
:100A3000C82AD92A6624C5C1E4E0F0E0CE2ADF2A1C
:100A4000C0C13FE3E32E7A94F3E6FF873CC1F20195
:100A500082E090E0480E591EE0807A9434C1F201A1
:100A600082E090E0480E591EA081B1817D01C3FE55
:100A700009C0862D992787FD9095BC01CD010E9464
:100A80003D081FC0FD0101900020E9F73197EA1BE6
:100A9000E88B18C0F20182E090E0480E591E0190E8
:100AA000F081E02D7F01C3FE09C0862D992787FDC7
:100AB0009095BC01CF010E94280803C0CF010E947D
:100AC0001F08888B9889791AFEC0C2FE0AC0F201FD
:100AD00084E090E0480E591E20813181428153818B
:100AE0000CC0F20182E090E0480E591E8081918195
:100AF0009C01442737FD4095542F79018A0157FF07
:100B00000CC0E2E0F0E0CE2ADF2A10950095F094C8
:100B1000E094E11CF11C011D111D8FEB9FEFC82219
:100B2000D92227C098E0988B08C0E0E4F0E0CE2AF4
:100B3000DF2AF8E7FF8720E1288BC2FE0AC0F20116
:100B400084E090E0480E591E20813181428153811A
:100B50000AC0F20182E090E0480E591E8081918126
:100B60009C014427552779018A01EFECFFEFCE2243
:100B7000DF22CE0101969A8B898B9889892E992440
:100B8000AA24BB24C801B701A50194010E947508DD
:100B9000DC01CB01E989FA8980838A3024F0FF8562
:100BA0008F0F815201C0805DE989FA898193FA8BA8
:100BB000E98BC801B701A50194010E94750879016C
:100BC0008A012115310541055105E1F6E98881E0E9
:100BD00090E08C0F9D1FE81AC60182739070892BDC
:100BE00009F07A94C6FE0DC0872D992787FD909550
:100BF000E889E03121F42EEF722E780E02C0782EB3
:100C00007A94C3FE0FC0262D332727FD30958E2DF5
:100C10009927821793072CF087EF9FEFC822D922DC
:100C200001C06E18C3FE02C0761801C07E18C6014E
:100C300080789170892B51F4872D7A94181634F4AA
:100C4000B10180E290E00E944808F6CFC1FE04C0E6
:100C5000B1018DE290E00BC0C4FE04C0B1018BE293
:100C600090E005C0C5FE05C0B10180E290E00E94A1
:100C70004808C6FE10C0B10180E390E00E94480819
:100C80009889903141F4B101EF858E2F992787FD26
:100C900090950E944808D0FE0AC0872D7A941816B5
:100CA00034F4B10180E390E00E944808F6CFC3FE1F
:100CB0000AC0862D6A94181634F4B10180E390E0DE
:100CC0000E944808F6CF90E8B92EBC2051F4872D39
:100CD0007A94181634F4B10180E290E00E9448083A
:100CE000F6CFFF85F33641F48E2DB101992787FDAC
:100CF00090950E94480840C02F852337B1F4888919
:100D00008150888B8F3FC1F1F70180810894E11CED
:100D1000F11CB101992787FD90950E944808988998
:100D20009150988B9F3F81F727C0EF85E33579F489
:100D3000F889F150F88BFF3FF9F0F7018491B10188
:100D400099270E9448080894E11CF11CF1CF6E011C
:100D50000894C11CD11C89899A898C159D0561F064
:100D6000E989FA898291FA8BE98BB101992787FD8C
:100D700090950E944808EFCFBB2069F0872D7A94A8
:100D800018164CF4B10180E290E00E944808F6CFBA
:100D9000B1010E944808CC24DD2413C09F85953200
:100DA00041F481E0C82ED12C6624762CEAE0E88B51
:100DB00008C0B101FF858F2F992787FD90950E946C
:100DC0004808F101838183FF04C0ED85FE85F4911D
:100DD00003C0ED85FE85F081FF872F85222309F072
:100DE0008BCDF1018681978162960FB6F894DEBFB4
:100DF0000FBECDBFDF91CF911F910F91FF90EF906C
:100E0000DF90CF90BF90AF909F908F907F906F902A
:100E10005F904F903F902F9008950F931F93CF9323
:100E2000DF93869F8001879F100D969F100D1124E0
:100E3000C8010E942907EC01009729F0A80160E091
:100E400070E00E943308CE01DF91CF911F910F9186
:100E50000895CF93DF93AC01029710F442E050E085
:100E600020E030E0A091B703B091B803BD01F901D3
:100E7000109709F44CC08D919C9111978417950798
:100E800031F14817590738F42115310519F0821747
:100E9000930708F49C01FD01A281B381109759F7D3
:100EA00021153105A1F1C901841B950B049708F4A4
:100EB000A901DB01E0E0F0E0109749F18D919C91F0
:100EC000119782179307F9F44217530779F4ED014C
:100ED0008A819B81309719F09383828304C0909319
:100EE000B8038093B703CD0102964AC0241B350B8B
:100EF000FD01E20FF31F41935193225030402D9397
:100F00003C93CF013DC0FD01A281B381D5CF80913B
:100F1000B5039091B603892B41F48091970190918C
:100F200098019093B6038093B503E0919501F091F9
:100F30009601309741F4EDB7FEB7809199019091F9
:100F40009A01E81BF90BA091B503B091B6039F017C
:100F50002A1B3B0B2417350788F0CA010296281775
:100F6000390760F0CD01840F951F02969093B60368
:100F70008093B5034D935D93CD0102C080E090E076
:100F8000DF91CF910895CF93DF93009709F454C078
:100F9000DC011297ED011B821A828091B7039091B8
:100FA000B803009721F1FC0140E050E0EA17FB078D
:100FB00018F1ED01FB83EA832D913C911197C20F4B
:100FC000D31FCE0102968E179F0771F48A819B81F1
:100FD000280F391F2E5F3F4F11963C932E9382812D
:100FE0009381FD01938382834115510559F4B09398
:100FF000B803A093B70320C0AF010280F381E02DB6
:101000003097A1F6EA01BB83AA83CA010296288120
:101010003981820F931F8A179B0771F48D919C91E0
:101020001197280F391F2E5F3F4F39832883FD0109
:10103000828193819B838A83DF91CF910895FC0104
:1010400005900020E9F7809590958E0F9F1F0895D9
:10105000FC010590615070400110D8F78095909583
:101060008E0F9F1F0895DC0140FF03C001C06D93E8
:101070006D9342505040D8F70895FC016150704084
:1010800001900110D8F7809590958E0F9F1F0895BD
:101090000F931F93CF93DF938C01EB018B819927E3
:1010A00081FF1CC082FF0DC02E813F818C819D81FC
:1010B0002817390764F4E881F9810193F983E883FB
:1010C00006C0E885F985802F0995892B39F48E8132
:1010D0009F8101969F838E83C80102C08FEF9FEF8F
:1010E000DF91CF911F910F910895A1E21A2EAA1BB3
:1010F000BB1BFD010DC0AA1FBB1FEE1FFF1FA217C8
:10110000B307E407F50720F0A21BB30BE40BF50BC4
:10111000661F771F881F991F1A9469F7609570954D
:0E112000809590959B01AC01BD01CF01089513
:10112E002A2A2A2A2A002A2A2A2A2A20466C617367
:10113E00682D4C45442070726F6772616D002A2ACB
:10114E002A2A2A204F757470757420777269747408
:10115E00656E20746F205541525431202A2A2A2A56
:10116E002A0A0052200042200059200025303278F1
:10117E002000433A20253032780A00526561643AE5
:10118E0020272563270A002A2A2A205072657373A6
:10119E002061206B657920746F20636F6E74696EA9
:1011AE007565002A2A2A20436F6E74696E75696E02
:0C11BE00672E2E2E000000B90320000058
:00000001FF
